:020000020000FC
:10000000D0CD00000000000020C0AEC18EC00000B6
:10001000000098C000000000000000000203040679
:10002000080C10182030406080000406080C1018DE
:100030002030406080A0C0000003070F1F000D0D9E
:1000400004050D050305030302004FB662FD0CC055
:10005000552041F00994C52DC095089483FDC7959E
:10006000C4BD64604FBE1895C0916400089483FDC0
:10007000C795C4BD6B7FC0916400CF3F09F41EC01B
:1000800070FF1AC082FD05C04FBE93989498959852
:10009000189576FD0EC065FD0CC0C091B100C0FD85
:1000A0009298C1FDC298C2FDC198CAEFC095CA9589
:1000B000F1F79398949895984FBE189524BCCC2747
:1000C000C064C8BF6460F8CFC6CF70FFC4CF65FD01
:1000D000C2CF939AC0CF70FFBECF65FDBCCF949ABC
:1000E000BACF70FFB8CF65FDB6CF959AB4CF929ACC
:1000F00070FFB1CF65FDAFCFC7E0CA95F1F7939A16
:10010000AACFC29A70FFA7CF65FDA5CFC7E0CA9559
:10011000F1F7949AA0CFC19A70FF9DCF65FD9BCF58
:10012000C7E0CA95F1F7959A96CF4FB6C9B7CF7E7B
:10013000C9BF6E7FCCB5CE0DDDB5DF1DDBBDCABD41
:100140004FBE18953FB68F7EA9B7A072A2118061ED
:10015000A9B7AF7DA9BFA9B7AE7FA9BF7894A09179
:100160006800AA2341F085FD2BC0A0916800AA95E4
:10017000A093680025C040E050E085FD15C0A6B3FF
:1001800096FDA095A0FD4FEFAEB5A06496FDAF7BA8
:10019000AEBDAA27A062A8BF8D7FA6B396FDA0958D
:1001A000A0FD5FEF451739F7A8E161FDA093680056
:1001B00085FD03C0A8E1A09368004093960081608C
:1001C00085FD0EC0A0916900AA2331F0A0916900BD
:1001D000AA95A093690004C08061AA27A062A8BF65
:1001E00080FF3CC0A09196004A2F61FF8E7F85FD65
:1001F0001CC0A091B400A430C1F4403F08F040EF0F
:10020000A42FA295AF704A0F5091B600533069F0F9
:10021000A695A69550FD01C0A69552FD03C0A41B4E
:100220004A2F03C04A0F08F44FEF40936100A72FF5
:10023000A670A1F073FD12C0A0917000AA0FAA0FC2
:1002400050919E0056955695541708F0452F4A0F29
:100250004093610018F4AFEFA09361004091B400A7
:10026000443009F03EC0A0916100A093630040912A
:100270006300A0919B004A1708F04A2FA0919D00AF
:100280004A1708F04A2F542EA091A000AA2309F47F
:1002900022C0542F5A1B10F4A42F50E0BA2E889479
:1002A000AA1FAA2EA091A200A095AA22A50E58F0DE
:1002B000A091A100A21509F0AA95AA0EA093A100F1
:1002C00048F04A2D08C0A091A100BA1608F0A395E5
:1002D000A093A1004FEF409364007F7B485F08F03C
:1002E0007064A52DA03408F06860A0916000A3950B
:1002F000A093600059F0F894A9B7A160A9BF84FF4A
:1003000003C0A9B7A062A9BF3FBE1895A091740011
:10031000A395A093740041E050916800552329F003
:1003200085FF03C05A9550936800A0919600A130B4
:1003300018F0209299000DC020929A002092A300FC
:10034000A0919900AF5FA093990018F0AFEFA09330
:100350009900F894A9B7A160A9BF84FF03C0A9B709
:10036000A062A9BF3FBE18953FB646B557B58F7E70
:10037000A9B7A072A2118061A9B7AF7DA9BFA9B723
:10038000AE7FA9BF789481FD25C0AEB5AF7B96FD49
:10039000A064AEBD8260A6B396FDA095A0FF05C087
:1003A000409365005093660041C1AEB5A06496FDD0
:1003B000AF7BAEBDAA27A062A8BF8D7F85FF01C01D
:1003C00028C140E0A6B396FDA095A0FD22C14093B0
:1003D000960011C1AEB5A06496FDAF7BAEBD8D7F1A
:1003E00061FF72C0AEB5AF7B96FDA064AEBDAA271B
:1003F000A062A8BF82604093910050939200A090A9
:100400008F004A19B09090005B09BB24A22C4C3895
:10041000520518F42092950049C0A091D400AA2357
:1004200059F1483C520528F4A0E1BA2EAAE0AA2EC0
:1004300023C04836A1E05A0728F4A8E0BA2EAFE05E
:10044000AA2E1AC0403DA2E05A0728F4A4E0BA2E12
:10045000AEE1AA2E11C0403AA5E05A0728F4A2E066
:10046000BA2EACE3AA2E08C04839A8E05A0720F4F7
:10047000A1E0BA2EA8E7AA2EC42EA0919300CA1A12
:10048000D52EA0919400DA0ADD202AF4AFEFC094B3
:10049000D094CA1ADA0A20929500A8E0A210A0E02F
:1004A000CA14DA0618F4A1E0A093950040939300D3
:1004B00050939400409191005091920040938F008E
:1004C0005093900042E097C0A09165004A1BA09114
:1004D00066005A0B94FD82C093FD80C092FD7CC0E3
:1004E00086FF03C0D52EC42E0CC05695479591FDAE
:1004F00073C05695479590FD6FC0D52EC42ED694E7
:10050000C79461FD19C0AC2DAC51AD2DA24008F0CF
:1005100005C0DD2089F4AC2DA85C70F4A0916700C3
:10052000A395AA2311F0A0936700AA3008F471C024
:100530002092960081606DC0A0916700AA2319F0F7
:10054000AA95A0936700A22C5091BA0097FD06C00F
:10055000A090C800533011F4A090D000AAEFAA0ECA
:10056000A22DA21DCA18DA0A4FB74170533049F4C0
:10057000442321F087FD05C0806803C087FF01C0C8
:100580008F77442359F0533031F4AFEFC094D094B7
:10059000CA1ADA0A03C040E050E020C0533049F4E0
:1005A000CC0CDD1CAAE0CA1AD20818F4A0E0CA2EAE
:1005B000D22CAFEFCA16D20418F04FEF50E00EC0A5
:1005C000A091AC00CA9E412D000C441F50E008F0E1
:1005D00012C04FEF50E00FC05695479594FF07C0EB
:1005E000552309F04FEFA42FA6954A0F521D4F3FF8
:1005F000520508F04FEF40939600816061FF09C0FB
:10060000AFE1A095A923AB299A2F8F7DBB2009F4D8
:100610008062A8E1A093680085FF03C0AAE0A093D0
:10062000680061FD03C085FD01C08F7E85FD03C0AC
:10063000A6E0A0936900F894A9B7A160A9BF84FFC0
:1006400003C0A9B7A062A9BF3FBE189511E00AC0B8
:1006500013E008C01AE006C01EE104C014E602C0A0
:1006600018EC00C005E1BB27BA95F1F70A95D9F758
:100670001A95C1F708952AE338E709C020E33CE85A
:1006800006C02AE234EB03C025E238EC00C012E0D9
:10069000BB27C29ABA95F1F7949ABA95F1F7949854
:1006A000BA95F1F7C298BA95F1F7123009F0939A1A
:1006B000123009F4959AB091AD00BA95F1F7123065
:1006C00009F09398123009F49598B7E8BA95F1F7C4
:1006D0001A95F1F6022FB22FBA95F1F70A95D9F7CC
:1006E0003A95A9F6C29A0895221B39E0001F3A955F
:1006F00009F40895221F211B18F4210F8894F6CFC6
:100700000894F4CF622C722CB0E08894B395221F29
:10071000331FE0F7379527958894912E802E020B92
:10072000130B10F4192D082D10F4889401C00894AF
:10073000661C771CBA9571F7172D062D0895322D7A
:1007400011232AF43A9500951095031B130BF89486
:10075000029F712C002D129F912C802C7894780C84
:10076000172D921C292DB4E06B2E26951795079511
:100770006A94D9F7332321F000951095031B130BCE
:1007800008950091B4000430A1F1B0919600B150E9
:1007900008F010C0B0916100B093630020927E0019
:1007A00020927F002092800020928100209282007F
:1007B0006F7B1FC06090B4006064B0916100B09323
:1007C000620008E317EC20917A0030917B003695A7
:1007D0002795B62DBA9541F036952795B62DBA9541
:1007E000BA9511F0369527958DDF00937E00109312
:1007F0007F00089500917E00B09162000B1B109164
:100800007F00120928F40038BFEF1B0740F009C031
:100810000F37120508F405C00FE710E002C000E82A
:100820001FEF0093830010938400089500918300CC
:10083000B09180000B0F10918400B09181001B1FBC
:1008400020E03091840033230AF42A95B09182008D
:100850002B1F1AF4203F40F00AC02F3008F407C0C5
:100860000FEF1FEF2FE003C000E010E020EF30910A
:100870006300B0919B003B1718F4323030F009C090
:10088000B0918400BB235AF004C0B0918400BB2314
:1008900032F4009380001093810020938200089529
:1008A0002091D70000918300000F10918400111F48
:1008B00046DF11232AF40038BFEF1B0740F009C0C0
:1008C0000F37120508F405C00FE710E002C000E87A
:1008D0001FEF002352F0B0916200B01B0B2F18F0F5
:1008E000013008F00AC001E008C000950F5FB09128
:1008F00062000B0F08F001C00FEF00938500089510
:100900002091D800009181001091820018DF1123FE
:100910002AF40130BFEF1B0740F009C00F3F12055A
:1009200008F405C00FEF10E002C001E01FEF112333
:1009300052F0B0918500B01B0B2F18F0013008F079
:100940000AC001E008C000950F5FB09185000B0F51
:1009500008F001C00FEF0093630008950FEF677F69
:1009600071FD29C072FD09C06860B0917B00BA308A
:1009700020F0B52DB03408F4677FB091D300BB23CD
:10098000D1F0B0917B00BB23B1F00FEF10917B0051
:10099000ABDEF894B091730072FDB5E00B9F112DA2
:1009A000002D7894112309F00FEFB0919E000B17E2
:1009B00010F400919E0000939D00089500917A002C
:1009C00010917B0000541140B0919D0010F4BA9535
:1009D00001C0B39511F0B0939D00089500C0089533
:1009E0002091B500B6B1B6FDFBCF04B115B1B6B1DB
:1009F000BF77B6B9B091AA00B395B093AA00B8304A
:100A000060F12092AA00B091D200BB2321F1112302
:100A100029F0B091AB00BF3F61F009C0B091AB00CD
:100A20000B1739F020F4BB2321F0BA9502C0B3951F
:100A3000E1F300919B00B093AB00B93B50F400ECA4
:100A4000BA3A38F400E8BB3920F400E4BC3808F4C2
:100A500000E000939B007F7E089510919B00B0E121
:100A60001B0F08F41FEF10939B00B091B400B4303B
:100A700081F000919B00B0916300B01B10F40091D5
:100A80006300B0919D000B1708F00B2F502E0093C0
:100A90006400B091AA00B73009F47061089502E3D0
:100AA000F894B091D9000B9F012D000C001F789491
:100AB000B0919B000B1710F000919B000093610018
:100AC00000936300502E0093640000939E000895ED
:100AD00020927A00B0EFB0937B000895F8940CB5A3
:100AE0001DB5209174007894309175006090760067
:100AF0000093750010937600031B160971FD03C067
:100B000077FD7DC027C0709077002093770027097C
:100B1000222311F00FEF1FEF809078009090790062
:100B20003093780060927900009175001091760002
:100B30000819190920917A0030917B003695279584
:100B4000020F131F10F40FEF1FEF00937A001093A2
:100B50007B0029C020917A0030917B003901B4E0FC
:100B60008B2EB2E09B2E343010F08A949A94383059
:100B700010F08A949A94769467948A94E1F72619EF
:100B80003709992021F0169507959A94E1F7200FDF
:100B9000311F20937A0030937B0028F43FEF30938D
:100BA0007A0030937B00323008F4706871FF02C025
:100BB000B3E00DC0B091C40000917100023838F06C
:100BC000B395003A08F0B395B63008F0B5E09B2E27
:100BD000B4E08B2E10917B0000917A0024E01695F2
:100BE00007952A95E1F70819120928F0B02FB2509D
:100BF000B12FB20910F402E010E0980126C0209154
:100C00007A0030917B0039017694679466946694FB
:100C100066942619320906950695200F321D2093F9
:100C20007A0030937B00323008F07F7704E036950D
:100C300027953695279526952695201B10F022306E
:100C400008F422E089019090C40060FDFECFE0909E
:100C50008B00F0908C006160B9B7B061B9BF38010A
:100C600077FD41C07694679400938B0010938C00BD
:100C7000B92DB330E1F0B0FD04C0060D171D93018E
:100C800006C0000F111F0250120922E030E0B92DFA
:100C9000B33068F020938D0030938E00009387006E
:100CA000109388006092890070928A003AC0009385
:100CB0008D0010938E0020938700309388006092FF
:100CC000890070928A0071FF0DC0BFE0B0938D0063
:100CD00020928E00B093890020928A00B0938B00FE
:100CE00020928C001EC0669400938B00B92DB33007
:100CF00091F0B0FD03C0060D262D03C0000F025079
:100D000022E0B92DB33038F020938D000093870096
:100D10006092890006C000938D0020938700609246
:100D2000890000917C0002FD0350013049F495FDDB
:100D300012C0B0B7B860B0BFB0E0B06CB7B90EC009
:100D4000023039F4B0B7B860B0BFB1E0B06CB7B939
:100D500005C095FDEECFB0B7B77FB0BF0091A20040
:100D6000000F10F4BBE60B270093A20060FDFECF3E
:100D7000B2E0B0936E006160B9B7B061B9BFB72F90
:100D8000B670D1F020917A0030917B00369527958E
:100D90003695279571FF02C0B0E43B0FF8940CB56F
:100DA0001DB5020F131F1BBD0ABD6160B0E1B8BFC6
:100DB000B9B7B061B9BF78940895606120927D00A1
:100DC00020E067FD20E206C0606120927D0020E205
:100DD00067FD20E001E011E077FD11C0B72FB6708C
:100DE00009F06F7E14E100917B00069509F40395EC
:100DF0000F3008F00FE071FF02C004E114E160FD64
:100E00000FC0B0917D00BB2359F071FF06C0B091B7
:100E10006E00BA95B0936E0011F4706249C0ABDFFA
:100E2000B0B73B2FB77FB0BFB8B1B0B733FDB86034
:100E3000B0BFB0917D00B395B0937D00B8B177FDA0
:100E400006C0B1E071FDB3E0BA95F1F7B8B1B07288
:100E5000B21709F022C071FF05C00395011708F011
:100E60000A95CDCF64FD05C00395011708F0B2CFF8
:100E7000C6CF6F7EF8943CB56DB470907A008090C8
:100E80007B00370D681C6BBC3ABD6160B0E1B8BF38
:100E9000B9B7B061B9BF78949DCFB0916D00B13052
:100EA00008F498CF64FD96CF0A9509F0A8CF7F7D0E
:100EB00020918D0030918E00F894B0E1B8BF0CB550
:100EC0001DB5020F131F1BBD0ABDE0908700F090F7
:100ED00088006160B9B7B061B9BF7894B72FB670B8
:100EE00039F0B0916D0072FFB395B0936D0009C0F9
:100EF00075FF07C067FD05C064FD03C0BF91BF91CA
:100F0000FCC4089500E063FF03C064FF01C001E07A
:100F1000F89410917100B7E01B9F212D102D78944B
:100F2000200F2695179526951795269517951093BA
:100F30007100183718F4B8E7B09371000091710090
:100F4000B09172000B1720F0606293989498959876
:100F500060FDFECFE0908900F0908A006160B9B733
:100F6000B061B9BF0895AC98B2E095FD0AC0F8949D
:100F7000B0937C00C29A929862FF01C0959A7894CF
:100F8000F9C0F894B0937C00C29AC19862FF01C086
:100F9000939A7894EFC0AC9AB3E082FF24C095FD99
:100FA00011C002E0F894B0937C00E1E8F0E0009317
:100FB000B1009598C19A62FF02C0949A01C0C2988C
:100FC0007894D8C002E0F894B0937C00E1E8F0E0B7
:100FD0000093B1009398929A62FF02C0949A01C064
:100FE000C2987894C7C095FD0BC0F894B0937C006C
:100FF000EBE6F0E0959862FF01C0949A7894BAC04D
:10100000F894B0937C00EBE6F0E0939862FF01C0A7
:10101000949A7894AFC0AC98B4E095FD0AC0F89467
:10102000B0937C00929AC19862FF01C0949A789420
:10103000A1C0F894B0937C00C19A929862FF01C05D
:10104000949A789497C0AC9AB5E082FF24C095FD3D
:1010500011C001E0F894B0937C00E7E7F0E0009362
:10106000B1009498C29A62FF02C0939A01C092980C
:10107000789480C004E0F894B0937C00EBE8F0E052
:101080000093B1009498C29A62FF02C0959A01C081
:10109000C19878946FC095FD0BC0F894B0937C0014
:1010A000E5E6F0E0949862FF01C0939A789462C0FC
:1010B000F894B0937C00E1E7F0E0949862FF01C0FF
:1010C000959A789457C0AC98B6E095FD0AC0F8940C
:1010D000B0937C00C19AC29862FF01C0939A789441
:1010E00049C0F894B0937C00929AC29862FF01C004
:1010F000959A78943FC0AC9AB1E082FF24C095FDE8
:1011000011C004E0F894B0937C00EBE8F0E00093A9
:10111000B1009398929A62FF02C0959A01C0C1985B
:10112000789428C001E0F894B0937C00E7E7F0E001
:101130000093B1009598C19A62FF02C0939A01C0D2
:101140009298789417C095FD0BC0F894B0937C00EA
:10115000E1E7F0E0939862FF01C0959A78940AC0A5
:10116000F894B0937C00E5E6F0E0959862FF01C04A
:10117000939A78946F7D089524E630E0F9012092E7
:10118000B100939894989598929AC29AC19A6B7F5D
:101190000895A2EBB0E009E00D9309E00D9304E09F
:1011A0000D930FEF0D9303E00D930FEF0D930AE0F6
:1011B0000D9303E00D9301E00D9301E00D93AEEB71
:1011C000B0E001E00D930FEF0D930D930D930D9390
:1011D0000D9303E00D930FEF0D930FEF0D930D9310
:1011E00005E20D9300ED0D9308E20D9300E50D93DC
:1011F00004E00D930FEF0D9302E00D9300E00D93CB
:101200000AE70D930FEF0D9300E00D9301E00D93AE
:1012100000E00D9303E00D9300E00D9308952091FD
:10122000B9008B7F233009F48460B091BA00B330E9
:1012300019F09F7DB1FD90629F7BB091BB00B1FD25
:101240009064223011F0886001C0877F08950A956C
:10125000E00FF21DB4910895ECE1F0E00091B200CE
:10126000F6DFB093D700ECE1F0E00091B300EFDFE0
:10127000B093D800EAE2F0E00091B800E8DFB09364
:10128000D9000091B800023008F402E00093730026
:10129000B091CE000FEFB23009F400EAB33009F498
:1012A00002E800937200E8E3F0E00091D500CFDFA0
:1012B000B093A000089508952091C8003091C9000E
:1012C000B091BA00B33009F43E5097FF02C020E05D
:1012D0003FEFB32FB21B6B2EB25810F4B2E86B2E57
:1012E00000E00395609EB12DBD57D8F30093AC008C
:1012F00008959068E1DFB0D920E030E0B0E16B2ED6
:10130000A7D9B09196002B0F321D6A94C9F7B4E0AB
:1013100036952795BA95E1F7822E9F77CDDF089510
:10132000F894E3E0F0E0B9E0B7BFB491B078C1F36E
:10133000F894A895B1B5B861B1BDB0E0B1BDB4E065
:10134000BEBFBFE5BDBF18DFB6E0B8BBB6E1B7BBF7
:10135000B8E0B5BBBCE1B4BBB4E0B2BBBCE3B1BB6D
:101360002224A0E0B0E02D92AA31E9F7A0E6B0E097
:101370000FEF2D920A95E9F7B1E0B093A20009DFD3
:10138000F8D2B7E0B06CB7B9B6B1B460B068B6B96E
:101390000091CA000093AD00B1E0B0936A00F894E8
:1013A0005FD969D959D96AD957D96BD955D9F89420
:1013B0000AEF1AEFA6B396FDA095A0FF1FC01A95DD
:1013C000C9F70A95B1F7E0E0FCE1B591B43E39F414
:1013D000B591B03E21F4B591BF3F09F40CC0E0E0F7
:1013E000F395F395B591B83F49F4B591B43931F41B
:1013F000B591BA3A19F4EE27F695099410DF2CDF6F
:101400005ADF5ADF0091CA000093AD00B5DEB2E0AA
:10141000B3BFB2E0BEBDB2E0B5BDB1E5B8BFB9BFC4
:10142000B0B70B2FB77FB0BFB8B1B0B703FDB8608E
:10143000B0BF0CD97894D2DA20927000BEB5B064F7
:1014400096FDBF7BBEBDB9B7B062B9BFBB27B06266
:10145000B8BF8D7F05D9626033E02CE0B091950074
:10146000BB2321F42CE03A9509F4A1CFF5D880FFF5
:101470009ECF8E7FB0919600B23078F3B92FBF71B6
:101480000091980000939700B0939800B01729F747
:101490002A9521F76D7FBEB5B06496FDBF7BBEBDBA
:1014A000BB27B062B8BF8D7FB091D400BB2321F4BD
:1014B0008062B92FB0709B2F8F7B20926700CED8AF
:1014C00085FF05C0B0916700BA3008F08064C0D8CD
:1014D00002E085FF01C000E0B0919600B017B8F3BC
:1014E000F894C9D8C8D8C7D87894BAD820928600BA
:1014F000B091BA00B33009F473C0AAD8B091BE005D
:10150000B13008F46DC0B0916A00B13008F468C021
:1015100085FD18C0B0919600BF3F08F461C0F894F3
:10152000B3D878949BD8B0919600B130C0F7F894B6
:10153000A2D890D8A0D8789491D8B0919600BF3F07
:10154000B0F3D8C2B3E09B2E9068F894B5DE7894DF
:1015500085D8F8949F77B0DE80909600B091960081
:10156000BF37789408F444C071D8F8948DD8789433
:101570009A9451F7BEDEB82DB093C90071D8F89493
:1015800025D28BD27894BAE09B2E9068F89494DEA2
:10159000789464D8F8949F778FDE80909600B0910D
:1015A0009600BF37789478F751D8F89464D852D819
:1015B00062D878949A9449F79CDEB82DBB5FB093BB
:1015C000C8004ED8F89402D277D2789447D8F894CD
:1015D00073DE7894B0919600BF3F08F499CF8AC229
:1015E00000919600B09186000B1710F000938600D2
:1015F00035D801E0B091BA00B35009F405E0B091DC
:101600009600B01708F074CFF8943ED83DD83CD877
:10161000789426D820926A0020926B0020926C0069
:10162000B0916B00B395B0936B00BF3F71F5B09173
:101630006C00B395B0936C00B091CC0009E1BA9501
:1016400059F002E3BA9541F00DE7BA9529F00AEF97
:10165000BA9511F020926C00B0916C00B017A8F010
:101660008BDDF4D7B0916C00BA95B0936C002092EA
:101670006B00B091CB00B093AD00F89405D878948E
:10168000B091CA00B093AD00E9D7E4D7B09168003B
:10169000BB2319F485FF01C08ACE01E085FD01C09E
:1016A00006E0B0919600B01708F4BACFB091BA0036
:1016B000B35009F0D3D7B0916800BB2309F477CEBB
:1016C000F8945ADD2092610020926200209263001B
:1016D000522C209264002092A1007894B091B7001F
:1016E000BB0FB0939F0020927E0020927F0020923B
:1016F000800020928100209282002092AA0060E067
:1017000070E020927100B8E0B093AA0070619ED79B
:10171000B7E074FDB6E0B06CB7B9B6B1B068B0640C
:10172000B6B9B6B1B6FDFDCF04B115B1B6B1BF774C
:10173000B6B9112309F00FEF0093AB0051D9B8E00F
:10174000B093AA0070616BDDF894BFEFB0939B007B
:10175000A6D9B0916100B0939B00B0939C00B09368
:101760009D007894B1E0B0936100B09363005B2E6C
:10177000B0936400B093A400B0919A00B093A3001A
:10178000B091BA00B33019F49F7D87FD906271600B
:10179000726020926D0097DCAEDC9AD99FD998D9FF
:1017A0009DD996D911DBEDD7ADDBDDDB97D905DB14
:1017B00066FD20D877FFD2D877FD00D9A3DBEBDB1D
:1017C0008DD902DB66FD32D89DDB25DC87D9F5DAC1
:1017D00066FD66D897DB37DC81D9F6DA66FD90D8EE
:1017E00091DB71DC7BD9E9DAB7E074FDB6E0B06C6F
:1017F000B7B9B6B1B068B064B6B984DB7CDC6ED979
:10180000EFD871FF24C0B0919E00B0939B00B093BD
:101810009C00B0919A00B093A300B1E0B093A400F3
:1018200018E12CE0B0916D00B11758F07D7F746025
:1018300020936F00B0919E00B0939B00B0939D00E9
:1018400006C0B0919600B13008F0ACCF60C072FF16
:1018500011C067FD0FC0B0916F00BA9519F47B7F7E
:101860007860A0CFB0936F00B0919600B13008F0CF
:1018700099CF4DC020927000B09199000AEF10915D
:10188000D600112309F003E0B01708F040C085FF2F
:1018900004C0B0916800BB23D1F1B091BA00B3305D
:1018A00081F495FD03C087FD04C00BC087FF01C014
:1018B00008C067FD06C06068B0919E00B0939B00B1
:1018C00086CF00EF67FF05C0B0919E00B0939B00EC
:1018D00000E2B0917B00B01708F464CF67FF17C037
:1018E0006F779F7D87FD90627460B2E1B0936F0067
:1018F000B0919E00B0939B0055CFB0917000B3950E
:10190000B0937000B0919600BB2309F002C0209202
:101910007000F89431DC8090B900B2E0B093B90067
:101920007EDC8092B90020926100209262002092B9
:101930006300522C2092640020929F0060E070E0CF
:1019400078948CD619DC0091D600002319F0939A74
:10195000949A959AB7E0B06CB7B9B6B1B460B06874
:10196000B6B985FF05C0B0917000B43008F01FCD46
:1019700053CEEDE0F0E023D0053509F01BC0EEE0DA
:10198000F0E01DD00A3A09F015C03AE0A2EBB0E051
:10199000E3E0F0E014D00D9331963A95D9F739E1B0
:1019A000AEEBB0E0EFE0F0E00AD00D9331963A955F
:1019B000D9F702C0EEDB0AD0E8E2F0E00895E19941
:1019C000FECFEEBBFFBBE09A0DB308951ED03AE008
:1019D000A2EBB0E0E3E0F0E00D910FD031963A9544
:1019E000D9F739E1AEEBB0E0EFE0F0E00D9105D0D2
:1019F00031963A95D9F712D00895E199FECF0DBBF3
:101A0000EEBBFFBBE29AE19A0895EDE0F0E00FEF44
:101A1000F4DFEEE0F0E00FEFF0DF0895EDE0F0E04E
:101A200005E5EBDFEEE0F0E00AEAE7DF089530914C
:101A3000AE000091AF00313011F40093B2003230AB
:101A400011F40093B300333011F40093B400343038
:101A500011F40093B600353011F40093B80036301D
:101A600011F40093C400373011F40093B9003830FA
:101A700011F40093D500393011F40093CE003A30C0
:101A800011F40093BA003B3011F40093BB000895A9
:101A900025E0E6D52A95E9F70895EDD5EFD5F1D5FE
:101AA000F3D5D8D5E8D5EAD5ECD5EED5D3D5E3D561
:101AB000E5D5E7D5E9D50895E7D5E3D5DFD5DBD57D
:101AC000C9D5E2D5DED5DAD5D6D5C4D5DDD5D9D5BB
:101AD000D5D5D1D508958090AE009090AF00CBD5EC
:101AE000CAD5C9D5B7D58A94D1F7CED5B3D59A94EE
:101AF000E1F70895F894D1DF7894CADFC9DFB1E047
:101B0000B093AE00B1E0B093AF002092B000F89473
:101B1000E2DF7894B5E06B2E70909600A1D5B0917D
:101B200096007B16C9F7B13018F0BF3F40F107C0EF
:101B30007EDFF8944BDFB1DFB8E0B1BDA9DF6A9476
:101B400059F7B091B000B395B093B000B33008F43A
:101B5000DECF9EDFB091AF00B395B093AF00F894A5
:101B6000B091AE00BA95EEE3F0E0EB0FF21D0491F8
:101B700078940395B091AF00B01708F4C6CF88DF12
:101B800087DFB091AE00B395B093AE00B091AE00D8
:101B9000BC3008F4B7CFFDDAF89418DFB8E0B1BD77
:041BA00077DFBECB62
:00000001FF
